:020000040000FA
:020000000928CD
:080008000B11950F0828960A60
:1000100009008501860183161130850000308600B5
:10002000FF30810083125C2259215C2251235C2223
:10003000AD210030AE00A02363220130AE00A0232A
:100040006322AD210230AE00A0236322AD21033034
:10005000AE00A02363220430AE00A0236322AD21B2
:1000600001220C3084008001840A30300406031D14
:1000700033281B21AD214630B1217230B1216530CA
:10008000B1217130B1213D30B1212030B1210B308F
:100090009A009B011A081C3E8400C3219A039A1FF0
:1000A0004A28073098005021AB308C0081018C0B1E
:1000B000572801088C0008309800031498038C0D11
:1000C000031C5E285021900191019201930181014E
:1000D00033218101921B31289401950196019701EA
:1000E000A0308B00FA308D00C7308C0000008C0BE4
:1000F00076288D0B74289301920130309100D53011
:1001000090003321810601088B019400921B312855
:10011000121315088C0016088D008E018F01031034
:100120008F0C8E0C8D0C8C0C10308400F72003107B
:10013000900D910D920D930D0310900D910D920D58
:10014000930D0310900D910D920D930D0310900DD2
:10015000910D920D930D9819B528980A0310940DDE
:10016000950D960D970D980BAE2800001030840069
:10017000DA200B309A0010088C0011088D0012084C
:100180008E0013088F009901990A14308400092108
:100190000318C42814308400F72099031A081C3E61
:1001A0008400190880009A039A1B392814308400AF
:1001B000DA20BB280310800D00088C00840A800D13
:1001C00000088D00840A800D00088E00840A800DCE
:1001D00000088F0084038403840303108C0D8D0DAD
:1001E0008E0D8F0D03108C0D8D0D8E0D8F0D0C0847
:1001F0008007840A0D0803180D0F8007840A0E0873
:1002000003180E0F8007840A0F0803180F0F8007CA
:1002100000340C088002840A0D08031C0D0F8002B4
:10022000840A0E08031C0E0F8002840A0F08031CA8
:100230000F0F80020034273084000008031D262998
:100240000408203A0319262984031D290430840256
:10025000053000070A300002031C00340A30800217
:100260000130840A292901088C00900F4429910F3C
:100270004C29920A013012060319121700000108D6
:100280000C06031D00343529121F4D290F301106AD
:10029000031D3F29921700340000000000003F2991
:1002A00018080F39F0388101640083168100831229
:1002B00000343030860083160030860083121430FC
:1002C00046227921053046227921013046227921C2
:1002D0007C212030860079212030AE210830AE21EB
:1002E0000130AE210630AE210C30AE210130AE21FE
:1002F00000348614861000348316F0308600831292
:1003000004308600861406088C0086108614861039
:100310008C1B8229860183160030860083120034EC
:100320008C018C038C0AF63E031892290A3E8C0E2F
:100330000C0708000F398C00093C3030031C073EC5
:100340000C0708008E000E0E9A21B1210E089A218A
:10035000B1210E0808008830AE2980308D007C2144
:10036000B4298D007C21083086000D08F039860400
:10037000861486100F3086050D0EF039860486141B
:1003800086100D0808000F3080051B1900349B08EB
:10039000031DD1291A08043A0319D1298008031929
:1003A00000340008303EB1219B0A1B19DC291523BB
:1003B000003A031DB12100342A23B1213723B12192
:1003C0004423B12100340008303EEB210023003AE1
:1003D000031DEB2100348C000508F6398C1A013816
:1003E0000C1B083885000C081F391B1C80389B1C0F
:1003F000403820388600DF398600203886009B0A86
:100400000034051C042A00348316DF308100831277
:100410009101920193018101A0308B00BE309500C3
:100420001008033903199503F0309600AD212030F0
:10043000B1214330B1214130B1214C30B1212030C4
:10044000B12113089021A2213A30B1211208902144
:10045000A2213A30B12111089021A221910A3C3009
:100460001106031D3F2A9101920A3C301206031D1A
:100470003F2A9201930A18301306031993011508B5
:10048000031D3F2A1608031D3F2A0E2A8D009530B2
:100490008C0000008C0B492A8D0B472A0134013057
:1004A000AF000130B0002030B100B10B552AB00BC5
:1004B000552AAF0B552A08000430AF001430B000A5
:0E04C0005630B100552A5C225C225C220800F6
:1006000003308A001A080F39820700346D34003431
:1006100000342E34003400344B34003400344D3474
:100620000034003447340034003403308A001A08A0
:100630000F39820700342E34003400342E34003455
:1006400000342E34003400342E34003400342E3480
:100650000034003403308A001A030739820700345B
:1006600000340034023402340234053405340330DB
:100670008A001A0307398207013401340134033434
:10068000033403340634063403308A001A0307396E
:1006900082072034203420340434043404340734F2
:1006A000073403308A004030AE218E010E08403AF4
:1006B000031900340E085F23B1218E0A562B8207DE
:1006C0000934093409340F34093409340934003445
:1006D000003400340F340234043408340F3400344E
:1006E0000834083409340A340C340A340934003428
:1006F0000934093409340F34093409340934003415
:10070000003400340F340234043408340F3400341D
:1007100008340D340A340A340834083408340034F8
:10072000143414341434173414341434143400349A
:100730001034103417341134123414341734003494
:100740002E0896000310960D960D960D960D9701A6
:100750001708160789008316081483120808003A40
:0E0760000319B62BB121970A171EA82B08000B
:084000000F000F000F000F007C
:02400E00F13F80
:104200004634723465347134413452345F34363458
:104210002E34413453344D3420342034203420346F
:104220003134363446343834343441342034513423
:104230003D34343420344D3468347A3420342034DE
:104240003234383420345334653470347434203488
:104250003234303432343434203420342034203476
:1042600020342034203420342034203420342034AE
:1042700020342034203420342034203420340034BE
:00000001FF
